:020000040800F2
:10500000881A0020D5500008FD8900080581000895
:105010000000000000000000000000000000000090
:10502000000000000000000000000000559600088D
:105030000000000000000000318F00086D9700089C
:10504000E7500008E7500008E7500008E750000864
:10505000E7500008C15B0008E7500008E75000086F
:1050600000000000E7500008E95A0008E750000877
:10507000E7500008ED85000800000000E750000838
:1050800000000000E75000080000000000000000E1
:10509000E750000800000000E7500008E750000853
:1050A000E7500008E7500008E7500008A5A10008F5
:1050B000E7500008E7500008000000000000000072
:1050C0000348854600F080FC00480047BDB7000853
:1050D000881A00200448804704480047FEE7FEE79E
:1050E000FEE7FEE7FEE7FEE709980008C15000086A
:1050F00030B50B46014600202022012409E00D4670
:10510000D5409D4205D31D469540491B25469540F7
:1051100040191546521E002DF1DC30BDF0B51FB40C
:105120000646002082B005464024019100901BE015
:10513000019922460F46304600F062FB049A059B17
:10514000801A994110D310461946224600F048FBB8
:10515000361A8F410197224601200021009F00F05E
:105160003FFB38184D4100902046641E0028DFDCCC
:10517000019B00982946324607B0F0BD03460B4319
:105180009B0703D009E008C9121F08C0042AFAD2FD
:1051900003E00B780370401C491C521EF9D2704783
:1051A000D2B201E00270401C491EFBD270470022BF
:1051B000F6E710B513460A4604461946FFF7F0FF16
:1051C000204610BD30B504460020034600E05B1CBD
:1051D000934203D2E05CCD5C401BF8D030BDF8B503
:1051E00002464A40D40F42004B0052085B089A42E4
:1051F00002D20246084611464A0023D0C30D4A0097
:10520000DDB2120EAD1A202D35DA49020126490A07
:10521000F6058A19002C00D0524220214F1B11465E
:10522000B9402A411018C20D9A4221D0002C17D043
:10523000012D08DCDA05801AD20F8019D207DBB203
:1052400000F00AFBF8BDDA05801A012340001B06B6
:10525000C01880185A428018CA0F1043490007E04E
:105260004908C2071143DA05801A801940088018DE
:1052700000F0EAFAF8BD61000122511A001BF7E7BD
:105280000122D2075140AAE70122D2075040A6E7E7
:1052900070B502464A40D50F40004A00ED0740086D
:1052A0005208002814D0002A12D0C40DD30D410298
:1052B0000120C0055202490A520AE41A09181218BC
:1052C0007D34914201D3641C00E04900002C01DAD6
:1052D000002070BD0023914201D3891A0343400886
:1052E00049000028F7D100290AD0914202D10121BA
:1052F000C90705E0914201D2012101E00121C94322
:10530000E005C018401900F09FFA70BDF0B50746DF
:105310000846584087B0C00F049048000E46590018
:1053200040084908BC1A884105D2384631461E4615
:1053300017460B4602465800400810434CD0300D2B
:10534000039040055900400D490D0590401A029008
:10535000402872DA18030121000B09050843019067
:1053600004980092002805D00199524200208841FB
:1053700000920190029840210A1A0199009800F0C9
:105380002FFA05460C466B4607CB00F04AFAC019C7
:105390007141039A0E0D0023D71756401A467A40E2
:1053A000164344D0049A002A2DD0029A012A039A67
:1053B00015DC1205C01A914101263605001C714109
:1053C000D20F059ED2070093019202962A462346E9
:1053D00000F088FA07B0F0BD38463146FAE7160506
:1053E000224A0F46B218C01AB74101210905001C14
:1053F0004F4100187F41114618187941E20F1043C0
:105400006D19644113E0E2076D0815436408C20793
:105410001443039A01261205C01A91413605001C57
:105420007141CE07400830434908C01851412A460F
:10543000234600F04AFACDE7FFE704980122400036
:10544000C117121A00238B4104983146C417381A29
:10545000A141EEE730B40124E407634030BC55E7D6
:1054600030B40124E407614030BC4FE70000E0FFA6
:10547000F0B51FB488B00B990998002448400999E9
:10548000C00F490049080991C0070B9900904900D5
:1054900049080B9109990898A64608431CD00B9916
:1054A0000A98084318D0099801244000420D48008A
:1054B000410D099824050003000B204309900B9827
:1054C0000003000B20430B9050181C494018002289
:1054D00001901446104605E0002001460DB0F0BDD5
:1054E000032801DA034600E003239C46C11A0AAEF2
:1054F0000AE05F0008ADED5B4F00F75B7D430027DE
:10550000AA187C41491C5B1E6145F2DD410004ABD9
:105510005A522104120C0A43240C401C0828DFDBD9
:10552000019802900099704601910090059B049AA1
:105530000799069800F0D6F9D0E700000DFCFFFFB0
:10554000F0B50C465C4085B0E40FE40703944C00D2
:1055500000266408590094464908024602962243F0
:1055600021D062460A431ED06200570D4A000E0346
:105570002303550D012402462C492405781B1B0BDF
:10558000360B401823432643614600901C46501AB0
:10559000B44103D30098401C009002E09218009898
:1055A0005B41002803DA0020014605B0F0BD002071
:1055B000012109050746864611E064461D46141B75
:1055C000B54106D36546521BB341744607430C43AD
:1055D000A646CD0740084908284392185B41054676
:1055E0000D43EAD11046184313D060461946504087
:1055F0007140084306D06046101AB34106D201221A
:10560000002306E000220123DB0702E00122D2434F
:105610005310009874460105381C6141029C039D9B
:105620000019694100F051F9BFE70000FD030000D7
:10563000C217C10F504010B54018CA079623002169
:1056400000F00AF910BD10B500229623114600F0B3
:1056500003F910BD0EB5C217C10F5040CA0740185C
:105660000021054B0293019200910A460B4600F07F
:1056700039F903B000BD0000330400000EB5054940
:105680000291002100910A460B46019100F02AF98F
:1056900003B000BD33040000410040020122400A73
:1056A000D205090E80187F2901DA0020704796295B
:1056B00003DC9622511AC8407047963988407047DB
:1056C00070B5CD0F4A0009030123090B1B051943CF
:1056D0000B4BED070024520D9A4201DA002070BDF9
:1056E000074B34339A4203DC9A1A00F089F802E03F
:1056F0000449511888402C43F1D0404270BD00004D
:10570000FF030000CDFBFFFF4A0009030123090B43
:105710001B051943094B10B5520D9A4201DA0020BE
:1057200010BD064B34339A4203DC9A1A00F068F835
:1057300010BD03495118884010BD0000FF03000050
:10574000CDFBFFFFC20FD207400040080BD0C10DB8
:105750000723DB01C91840020905400A1143C208AA
:1057600040071143704700200146704710B50029DB
:1057700004DB0124E40740428C412146002B04DB7A
:105780001C460123DB075242A341994200D19042BB
:1057900010BD0000CB0FDB07490010B549080246D9
:1057A0000A4307D00A0D07240903E401090B121B61
:1057B000002A01DC002010BDC900440F0C43C100C9
:1057C000E018D205801800F03FF810BD0122D20782
:1057D000002800DB101A002900DB511A81427047B3
:1057E00010B5202A04DB0146203A9140002010BD6C
:1057F000914020239C1A0346E3401943904010BD7A
:1058000010B5202A04DB0846203AD040002110BD04
:105810000B46D340D0402024A21A91400843194699
:1058200010BD10B5202A06DBCB170846203A1041E0
:10583000C1170B4306E00B461341D0402024A21AA7
:1058400091400843194610BD002904DA401C490064
:1058500001D140084000704770B40024050C05D108
:105860001024000402D1002921D01124050E01D1F9
:1058700000020834050F01D10001241D850F01D15C
:105880008000A41C002801DB4000641C002908D013
:1058900020252E1B0D46F540A14000D001212943B3
:1058A000084301061B1B000ADB1D02D5002070BC4B
:1058B0007047DB05181880180029F8DA401C4900E9
:1058C000F5D170BC40084000704710B5002B08DAD5
:1058D0000024401C614192185B411A4301D14008E9
:1058E000400010BDF0B51FB482B005460C0003D0D7
:1058F000084604F017FD02E004F014FD20300246D3
:10590000009021462846FFF76BFF049B059A04464A
:105910000F4618431143084314D0184610431BD0B8
:10592000009840210A1A18460599FFF769FF0546B5
:105930000E46009A05990498FFF752FF084305D0D8
:10594000012004E02046394607B0F0BD0020C11711
:1059500005430E432C43374300990E986305401AC4
:105960007905E40A00220C43FD0A0A3002D5002022
:105970000146E9E70105101969410C9C0D9D0019CC
:105980006941FFF7A2FFDFE74A0009030123090B82
:105990001B0519430A4B10B5520D9A4202DA00203A
:1059A000014610BD064B34339A4203DC9A1AFFF7C6
:1059B00027FF10BD034BD218FFF712FF10BD0000E8
:1059C000FF030000CDFBFFFF064C0125064E05E05E
:1059D000E36807CC2B430C3C98471034B442F7D310
:1059E000FFF772FB40BB000860BB000870B58C1865
:1059F0000578401C6B075B0F01D10378401C2A110E
:105A000006D10278401C03E006780E70401C491C49
:105A10005B1EF9D12B0705D40023521E0DD40B7049
:105A2000491CFAE70378401CCB1A921C03E01D784E
:105A30000D70491C5B1C521EF9D5A142D8D3002021
:105A400070BD000038B50446064805490068FFF7F8
:105A50004FFB604300E0401E00900028FBD138BDA2
:105A600040420F0028010020F8B504460068816814
:105A70008907890F012902D10168C90722D18168EC
:105A8000114A10261140012500290ED181682943B1
:105A900081600120FFF7D6FF00F0A4FF07460CE06D
:105AA00000F0A0FFC01B0A2807D9606D3043606575
:105AB000A06D2843A0650120F8BD20680068C043A0
:105AC000C007EDD10020F8BD1700008010B50023FD
:105AD0001A4603E0845CE3189BB2521C8A42F9D355
:105AE000D84380B210BD000010B5034800F036FD69
:105AF000024800F033FD10BD28160020E0150020FC
:105B000030B5446C1C252C400125A540046C656013
:105B1000046863608368102B036803D09960006891
:105B2000C26030BD9A600068C16030BD1449012078
:105B300048720A4602205E32507203203C3A50728C
:105B400004200E3A50720F480D4B00780870223135
:105B50000870203108770C495A1C08785871497828
:105B6000997123331871597120331877597710754B
:105B700051751A461E321075517510765176704760
:105B80005C110020D7000020F800002010B503F0C1
:105B900037FD202003F0E0FD012005F069FB002027
:105BA00003F0DAFD044805F007FA044805F0B6FCF6
:105BB000002005F0EBFC10BDC00000208380000039
:105BC000F8B505200121000700F0F8FE0025174C6C
:105BD000002800D06560164E0221304600F0EEFE2F
:105BE00000281BD1012020701248808F00280ED081
:105BF0000127BF0200223946304600F0ECFE0A20A1
:105C000005F08CF901223946304600F0E4FE0A48DE
:105C1000656000880A21484308490880012000F097
:105C200005FE022000F002FEF8BD00001401002075
:105C3000000400505C0D0020E4000020F60000206D
:105C40007047000010B5084900224A6107494B68B7
:105C50004C1523434B604B68082423434B60C00919
:105C6000C001026010BD000070160020002002403C
:105C70007FB500250C460646039500F0A7FDE00918
:105C8000029003A901960095684600F037FD0028B0
:105C900004D000F06FFD002004B070BD00F06AFD7C
:105CA0000120F9E710B5002302E0C45CCC545B1C72
:105CB0009342FAD310BD000010B5214A002190692B
:105CC000C305204804D54169022319434161911558
:105CD00093699B0505D5436901242343436163020E
:105CE000194393695B0505D5436908242343436140
:105CF000E301194393691B0505D543690424234334
:105D000043616302194393699B0405D543691024D9
:105D1000234343616302194393699B0304D5446998
:105D200020231C43446119439369DB0305D5436970
:105D3000402423434361A0020143916110BD000050
:105D4000002002407016002070B5054600F04AFEA3
:105D50000646184C0AE0681C08D0002D04D000F05C
:105D600041FE801BA84201D9032070BDA069C00775
:105D7000F1D1A069800701D50220A061A069C0050A
:105D800011D4A06980050ED4A06940050BD4A06988
:105D9000000508D4A069800405D4A069800302D45A
:105DA000A069C00303D5FFF787FF012070BD002065
:105DB00070BD000000200240F8B5174600260546D9
:105DC0000C4600F003FD09E029460220226800F09D
:105DD000DFFC002804D1241D2D1D361DBE42F3D347
:105DE00000F0C8FCBE4201D20020F8BD0120F8BD81
:105DF00010B5084902460020054B497905E04400EA
:105E00001C5B944203D0401CC0B28842F7D310BD43
:105E1000841200205800002010B500F0D4FD10BD01
:105E200010B5094800F0F2FF80B2FFF727FC074ADF
:105E3000074BFFF71DFB0022064BFFF781FBFFF727
:105E400063FC80B210BD000094140020F853E3A559
:105E50009B843E4000408F4070B5354C3348217FD5
:105E60000175617F417533490A7802764978417638
:105E70002E490520133148720A2005F03FFB7D2092
:105E8000C00005F055FB2949002213310C2005F014
:105E90001FFC00210C2005F02DFC022005F07EFBEC
:105EA000254D00210F2005F0A9FA2842E062F8D024
:105EB000E06A411C38D0400435D58122D20100214E
:105EC0000F2005F0DAFB0021102005F097FA4106BB
:105ED0001648490E0022633005F0C6FA134D6335AB
:105EE000687A05281FD102221249681DFFF76AF956
:105EF000002818D10E48AE7C66710422691C40301F
:105F0000FFF73CF929461331084672000D4651301F
:105F1000FFF734F96079294642000448DF30FFF783
:105F20002DF90320207070BD04F05AFABD11002035
:105F300058000020F800002000D0272410B50848A1
:105F400000F096FA0A21064800F032FA044800F000
:105F50001DF9800503D5024800F01AF980B210BD82
:105F600038140020F8B52F4D00220121284600F0FA
:105F700032FDFFF7E3FFFFF766FB2B4E3146FFF7DD
:105F800087F92A4C0122A0601146284600F023FD23
:105F90002749A068002588423EDB2078254F00284D
:105FA00015D02570FFF7CAFFFFF74DFB3146FFF70D
:105FB0006FF9A060FFF7C6FB00223B46FFF74AFAE5
:105FC00000221D4BFFF754FAFFF7E4FB6060A06866
:105FD000FFF7B8FB00223B46FFF73CFA174A184B85
:105FE000FFF746FA06460F466068FFF7ABFB134A19
:105FF000144B5242FFF73CFA32463B46FFF786F914
:10600000FFF7C8FB10496060884201DD616004E071
:10601000FF21C905C84200D365606068FFF73CFBFB
:10602000C0B2F8BD0004005000401B443000002006
:106030000000604000000C4000E064403333333324
:1060400033B33040CCCCEC3F0000C842F8B5054635
:1060500004464035287C0026012808D001202874F9
:10606000206881688907890F01290ED101E002208B
:10607000F8BD0168C90708D0606D2021084360653C
:106080000126002028743046F8BD616DFF220132E0
:106090009143022211436165C1688907890F00910C
:1060A000C16889088900C16020688168920711432E
:1060B000816000F097FC07460EE000F093FCC01BE7
:1060C0000A2809D9606D02218843102108436065C0
:1060D000002028740120F8BD206880680028ECDBCF
:1060E0002068C168009A1143C160606D800880001B
:1060F000401C6065C5E70000F8B506460D46403611
:10610000317C01290DD00121317401688A68520760
:1061100009D5416D202211434165002030740120D2
:10612000F8BD0220F8BD174B6A68D80547109A429F
:10613000154C8A6A2B6812D05B035B0B1A438A6288
:106140002968490305D5A1680143A1600A20FFF72A
:1061500079FC2868800312D5A06838430EE05B0301
:106160005B0B9A438A622968490302D5A16881437F
:10617000A1602868800302D5A068B843A060002011
:106180003074F8BD0110000000270140406D7047D9
:106190000068006C7047000070B5040006D0606DA8
:1061A000264600254036002802D006E0012070BDBA
:1061B000A5653574204600F0D3F8606DC00603D4A1
:1061C00021688868400705D5606D10210843606527
:1061D0003574EBE7606DFF220132904302221043D9
:1061E000606588688207920F5B48012A02D10A68BD
:1061F000D2072BD1032362689B079A4205D05B42EA
:106200009A4202D05B009A4209D10A699200920830
:106210000A6121680A6963681A430A610CE00A6925
:10622000920092080A6181680F2292049143816072
:1062300081686268114381602168CA6818239A43A3
:10624000CA602168CA68A3681A43CA6081680122CB
:106250005206914381608168A28E5206114381608B
:1062600020688168C90004D48168012212071143A3
:1062700081602068C168394A1140C1602069E168C5
:10628000022825D000200143204620300278037BDD
:1062900052035B001A431143226B1143A26992031C
:1062A0001143E269D20311432268D3681943D160D4
:1062B000616A0A46FF3AC23A05D0A26A11432268CF
:1062C000D3681943D16042780121012A02D00BE042
:1062D0000420D8E70078002823D0606D20221043E6
:1062E0006065A06D0843A065E06B012820681FD0A1
:1062F0000169C90703D001694908490001612068A3
:106300004169C908C900416120684169A26B114314
:106310004161A565606D80088000401C60650020BB
:1063200070BD2068C26801231B041A43C260DBE70A
:106330000269FF239B009A43026120680269236C73
:10634000A66C1A43636C33431A43026120680269E6
:106350000A430261D3E70000002701401902FEFF53
:1063600010B586B0044614216846FEF720FF0E499A
:106370002068884216D10D48416B42151143416394
:10638000C16A01221143C162C06A6946104005908A
:1063900002200090032001900020029005200007B9
:1063A00000F050FA06B010BD002401400010024079
:1063B000F8B504464069254640350E4608280BD0FE
:1063C0002068C068C00709D0606D2021084360655F
:1063D000002028740120F8BD082700E00C2700F0F9
:1063E00001FB009011E0701C0FD0002E05D000F0D2
:1063F000F9FA0099401AB04207D9606D04210843A8
:106400006065002028740320F8BD206800683842C9
:10641000E9D0606D01214902084360652068C168C8
:1064200009058A0F0C21002A1BD12022125D002AA7
:1064300017D10268120714D5826853070122002B76
:1064400008DB43688B434360606D1302984310433D
:10645000606506E0606D202318436065A06D104301
:10646000A065A069002801D1206801600020F8BD66
:1064700070B50446216800208968490721D4254663
:106480004035297C01291CD001212974E1690129A9
:1064900004D02046FFF7E8FA002811D1616D0A4ABE
:1064A0001140FF220132114361650021A165297469
:1064B00022681C21116021688A6804231A438A60BB
:1064C00070BD022070BD0000FEF1FFFF30B5014637
:1064D00020314A790023022A04D00422C2630B71BE
:1064E000012030BD026814680E25AC4314600268B8
:1064F0001468640864001460446C1C221440012277
:106500001546006CA54045604A7118460B7130BDB8
:1065100070B50024014620314A79022A03D00421B3
:10652000C163012418E0026813680E25AB431360B1
:10653000026813685B085B001360436C1C22134005
:10654000012215469D40036C5D604A7100220A716C
:10655000816B002900D08847204670BDF0B4016CE3
:106560000D6801680C68466C1C2304221E40174607
:10657000B7402F420ED067070CD50C68A40602D492
:106580000C6894430C60416C19408A40016C4A606D
:10659000016B1AE00227B74002462F402032002F3D
:1065A00017D0A70715D50C68A40605D40C680A25D2
:1065B000AC430C6001215171446C02211C40036CFE
:1065C000A140596000211171C16A002918D0F0BCA6
:1065D00008470827B7402F4212D0240710D50C686F
:1065E0000E25AC430C60446C01211C400B46A340BB
:1065F000046C6360C163517100211171416BE4E768
:10660000F0BC704770B504003CD01F4825681421C9
:106610002818FEF76DFD800060641C48206402218C
:10662000204620300246417129681948E36801403C
:10663000A06866691843236933431843A369184364
:10664000E3691843236A1843084328600121A068BE
:106650008903884210D00D488030836A656C1C2104
:106660000D400F26AE40B3438362656C63680D40F6
:10667000816AAB400B4383620020E06301215171CA
:10668000107170BD012070BDF8FFFDBF0000024019
:106690000F80FFFFF8B504468C46203001790025B5
:1066A000012909D00126067141790027012905D069
:1066B000077102252846F8BD0220F8BD022141716C
:1066C000E763206801684908490001606146204687
:1066D000FFF716FA206B00282068016801D00E220F
:1066E00005E0042291430160206801680A221143F9
:1066F00001602068016831430160DBE7F8B51A4E9C
:106700000546307C0F46012807D001203074174819
:10671000FFF71AFB010002D021E00220F8BD0020A3
:10672000C04338606C6814E02046FFF78BFA0F48CE
:10673000FFF70AFB01460E48426808239A4342606D
:10674000426843159A434260002901D03C6006E04C
:106750008034A8686A68C0018018A042E4D800208C
:1067600030740846F8BD00007016002050C30000C9
:1067700000200240054841680222114341604168FF
:1067800001221143416000207047000000200240B8
:10679000F8B50C4C1646207C0F46012808D0012085
:1067A00020740948FFF7D0FA0025002802D006E03F
:1067B0000220F8BD65613E600348FFF7C5FA257405
:1067C000F8BD00007016002050C300001148416859
:1067D000C9070BD0EFF3108172B60F4AC2600F4A9F
:1067E000C26081F310884168C9070ED141688907EA
:1067F0000DD5EFF3108172B6094A0261094A0261B0
:1068000081F310884068800701D50120704700207F
:106810007047000000200240EFCDAB890504030261
:10682000BFAE9D8C161514137047000010B50449B7
:106830004A69024202D04861FFF7F6FF10BD00002E
:1068400000040140FCB500230124A2E027462A46AB
:106850009F403A406FD04D68012D05D0022D03D0E6
:10686000112D01D0122D16D185680326AC465D008E
:10687000AE46AE406546B543AC46CE687546AE40C2
:1068800065462E43866046680D79BE43ED06ED0FE2
:106890009D4035434560C6685F000325BD40AE4658
:1068A000AE4335468E68BE402E43C6604E68022E0B
:1068B00001D0122E14D1DE08B60036180196366AC1
:1068C0005D07B446EE0E0F25B54000966646AE4312
:1068D000B4460D69009EB54066462E43019D2E626A
:1068E00006687546AE430D79AD07AD0FBD40354323
:1068F00005604D68ED004BD5294D6E6B26436E63E8
:106900009E08284DB6007519AC46AD689E07360F37
:106910000F27B740BD4305273F07B84201D10027E5
:1069200015E0214FB84201D1012710E01F4FB842B6
:1069300002D102270BE02BE01D4FB84201D1032703
:1069400005E01C4FB84201D1052700E00627B740FB
:106950002F436546AF60184D2E684F689643FF037E
:1069600000D516432E606E684F689643BF0300D56E
:1069700016436E60AE684F689643FF0200D516431B
:10698000AE60EE684F689643BF0200D51643EE60D6
:106990005B1C0A681546DA4000D057E7FCBD0000D2
:1069A00000100240000001400004005000080050A8
:1069B000000C0050001C0050000401400069084019
:1069C00000D001207047426913460B401B049143DD
:1069D0000B4383617047002A01D081617047816257
:1069E0007047000001488068704700001C010020CB
:1069F0000248816802788918816070471C01002074
:106A000010B5084800240168402211430160204667
:106A100000F00AF8002801D0012401E000F040FA5B
:106A2000204610BD0020024070B504460D4D7D206B
:106A30002978C000FEF75CFB01460B480068FEF7B2
:106A400057FB00F029FF002809D1042C07D20022AF
:106A50002146401E00F04CFA00206C6070BD012001
:106A600070BD00001C010020280100207047704705
:106A7000F8B55E4CA078401CA07001202071A08B5E
:106A8000401CA0835A48008802F022FE594DE88835
:106A9000FEF7D9FD5849FEF7FBFB584E0746316813
:106AA000FEF79DFB30600120A16AC005814203DB37
:106AB0003846FEF7E9FBA062607800280CD102217D
:106AC0004F48FFF77BFF02004E494F4817D0002286
:106AD000FFF781FF0020A06302214948FFF76EFF06
:106AE0004A4F002852D00020A063A88AFEF7ABFDD1
:106AF000424E3168FEF76AFE59D2012058E0012269
:106B0000D1034148FFF767FFE888FEF79CFD3A494B
:106B1000FEF7BEFBA16BFEF762FB3D49A063884216
:106B2000DADD34480127F926403000900A2130464A
:106B3000FEF7DEFA002903D132493348FFF76CF93A
:106B400002212F48FFF73AFF002801D0002701E07B
:106B5000002F12D102212A48FFF730FF00280CD164
:106B600004F000FF00990120888004F059FF6420A0
:106B700004F0D4F928492748C8600A2004F0CEF967
:106B80003046761EF6B20028D0D1A5E7E888FEF799
:106B90005AFD1949FEF77CFBA16BFEF720FB1F494C
:106BA000A0638842A1DB1C491A48C8609DE7002009
:106BB0003870688F401EFEF73BFD3168FEF706FE19
:106BC00004D86079002801D0012000E00020144999
:106BD0000870688FFEF737FD3168FEF7F7FD04D2C5
:106BE0006079002801D004F081FEF8BDD4000020B7
:106BF000720000205C0D002000007A441801002083
:106C00000004005000800000000000505E000020E2
:106C1000000040400400FA0500ED00E00000A04044
:106C20006B000020704770B5040010D0022025468C
:106C30002035A873204601F0E1FCA87B032805D08D
:106C4000204600F0B9F80020A873687370BD0120D9
:106C500070BD7047704710B5044600680168C943AD
:106C6000C90708D18168C943C90704D1012141601E
:106C70002046FFF7FDFE20680168C943890708D454
:106C80008168C943890704D4022141602046FFF787
:106C9000EDFE20680168C943490708D48168C943EB
:106CA000490704D404214160204600F0F7F8206829
:106CB0000168C943090708D48168C943090704D496
:106CC000082141602046FFF7ADFF20680168C943F5
:106CD000C90608D48168C943C90604D4102141609B
:106CE0002046FFF7C4FE20680168C943890608D41E
:106CF0008168C943890604D4202141602046FFF7FA
:106D0000A9FF20680168C943490608D48168C943BE
:106D1000490604D4402141602046FFF79AFF10BD88
:106D2000F8B5040005D025462035A87B002802D000
:106D300006E00120F8BD00206873204600F04EF800
:106D40000220A8732068C26884466368012B01D1C1
:106D50000620824316486169814202D00720400321
:106D60008243002B01D1D82082431248A6680240FA
:106D700018463043676A266A3E433043A66A30436A
:106D80001043002B02D0012B04D005E02369E269F7
:106D90001A4300E0E2681043054A914202D0A2691A
:106DA000114308436146C8600120A8730020F8BD64
:106DB000FFFF0000F8F119FF10B50068054988428F
:106DC00007D10548816B4900490881630D2000F017
:106DD00073F810BD007C00400010024010B5006840
:106DE000084988420CD10848816BC2041143816371
:106DF000002201210D2000F07BF80D2000F06CF83E
:106E000010BD0000007C0040001002400068C06916
:106E100070470000F8B50446022025462035174685
:106E2000A8731D480268C3041A4302602068C26840
:106E30009B121A43C2602068026901263243026134
:106E4000226810205060206881611021204601F0E6
:106E500045FC03281FD0216808204860206847614E
:106E60000821204601F03AFC032814D0204601F006
:106E7000C5FBA87B03280ED0206881683143816060
:106E800020680169314301612068016904221143CE
:106E90000161AE730020F8BD00040140704700009E
:106EA0000448416B012211434163816B0204114389
:106EB0008163704700100240002809DBC106C90E3B
:106EC0000120884003490860BFF34F8FBFF36F8FE5
:106ED0007047000080E100E0002805DBC106C90E14
:106EE00001208840014908607047000000E100E08F
:106EF00010B503F053FA10BD02494A6882434A6054
:106F0000704700000070004002480168821511437C
:106F1000016070470070004002494A6802434A60BD
:106F200070470000007000400548016802221143CC
:106F300001600448016904221143016130BF7047B8
:106F40000070004000ED00E0F0B5154A1368154DE3
:106F500054152D6A2340ED07ED0F002B04D0002DB2
:106F600002D01668A64316601668B608B600064337
:106F700016600D48076904263743076101290DD0C3
:106F800040BF20BF20BF0169B1430161002B04D085
:106F9000002D02D0106820431060F0BD30BFF2E732
:106FA000007000400000014000ED00E0F8B504462C
:106FB00000780027534D800671D5524E403EB06B8D
:106FC000C00004D4B06BA9050843B06301274E4844
:106FD0000168C90511D40168821511430160FFF7EA
:106FE00001FD009005E0FFF7FDFC0099401A6428C0
:106FF00037D845480068C005F5D532680321090532
:1070000060680A400140914208D08103890F03293A
:1070100004D13168890301D50120F8BD2A69032113
:1070200009040A4022D0084090421FD020788006F0
:107030001CD528692A6988430121C9040A432A61A9
:107040002A698A432A612861C0050FD5FFF7CAFC67
:10705000009008E0FFF7C6FC0099411A2B488142D6
:1070600001D90320F8BD28698005F3D5616888033C
:10707000800F032805D132680005824301400A438E
:1070800032602869032261681204114008432861B4
:10709000002F04D0B16B012000078143B163207839
:1070A000C00705D0E868A168800880000843E86050
:1070B0002078800705D5E8680C218843E1680843FB
:1070C000E8602078400706D5E868032189028843F4
:1070D00021690843E8602078000706D5E8680321A5
:1070E0000903884361690843E8602078000606D5F3
:1070F000E868032189048843A1690843E860002007
:10710000F8BD0000401002400070004088130000ED
:10711000F8B50E46050038D05E480068C007C00FBD
:10712000B04214D25B4C20684008400030432060DD
:10713000FFF758FC074605E0FFF754FCC11B564813
:1071400081427AD82068C007C00FB042F4D12878B5
:10715000524C800705D5E068F0218843A9680843B0
:10716000E0602878C00752D06868022806D003285B
:1071700007D0216801280AD0890504E02168890325
:1071800001E021688901002903DB0120F8BD4907DE
:10719000F9E7E168890889000143E160FFF722FC13
:1071A0000746686802280AD0032814D001281ED098
:1071B00029E0FFF717FCC11B374881423DD8E06842
:1071C0000007800F0228F4D121E0FFF70BFCC11B60
:1071D0003148814231D8E0680007800F0328F4D19C
:1071E00015E0FFF7FFFBC11B2B48814225D8E06863
:1071F0000007800F0128F4D109E0FFF7F3FBC11B62
:107200002548814219D8E0680007800FF5D1214850
:107210000168C907C90FB14217D901684908490077
:1072200031430160FFF7DEFB074608E005E0FFF7AA
:10723000D9FBC11B1848814201D90320F8BD15486C
:107240000068C007C00FB042F1D12878400706D5CA
:10725000E068072109028843E9680843E06028786C
:10726000000707D5E0680721C90288432969C900DA
:107270000843E06000F03AF8E168094A0906090F9E
:10728000515CC8400749086007480068FFF7CCFB1D
:10729000F8BD0000002002408813000000100240EA
:1072A0001EBB0008280100202001002004480549D9
:1072B0000068C968044A4905490F515CC8407047D5
:1072C000280100200010024037BB0008044805498F
:1072D0000068C968044A8904490F515CC840704776
:1072E000280100200010024037BB000870B51A4A80
:1072F000D3681A490C2018408D0004280CD04E0089
:10730000082810D00C2810D050680004410F01202C
:10731000C003491C884070BD1068C00601D50846EE
:1073200070BD284670BD304670BD98020C4C000FF1
:10733000205C1B029C0FD368641CDB0301D5314623
:1073400003E01268D20600D4294603F002F8224670
:107350000023FDF7E3FE70BD0010024000093D0070
:107360002EBB0008FEB505007ED0FE4CE7680C2061
:10737000E66807400120000406402878C00747D08F
:10738000082F05D00C2F0AD101200004864206D117
:10739000206880033CD568680028E5D038E00120EB
:1073A00069680004814203D121680143216011E032
:1073B000052301221B0492049942216802D1114342
:1073C0002160F1E78143216021680140009120683C
:1073D00090432060686800280DD0FFF703FB009001
:1073E00005E0FFF7FFFA0099401A64287BD820686F
:1073F0008003F6D50CE0FFF7F5FA009005E0FFF703
:10740000F1FA0099401A6428F0D820688003F6D475
:107410002878800756D50923E868042F0DD00C2F53
:1074200001D1002E09D000283CD0216899430143A6
:107430002160FFF7D7FA064628E02168490701D501
:10744000002891D061681F22120291432A6912021A
:10745000114361602168994301432160FFF746FFB2
:10746000E16809060A0F00E08BE1BF49895CC8406A
:10747000BE490860BE480068FFF7D6FA002873D1FD
:1074800020E0FFF7AFFA801B0228AFD82068400742
:10749000F7D560681F21090288432969090208435A
:1074A00060600FE02068400840002060FFF79AFA13
:1074B000064604E0FFF796FA801B022896D820685B
:1074C0004007F7D42878C00660D5002F0CD0A869F3
:1074D00000284AD02068FF21013108432060FFF7CF
:1074E00081FA06462EE0C1E02068800502D5A86931
:1074F0000028A6D06068072149038843296A084309
:1075000060606068297F0002000A09060843606025
:10751000286A410B0120C003491C8840E168090624
:107520000A0F9149895CC8409049086090480068FA
:10753000FFF77AFA002817D128E0FFF753FA801BEB
:107540000228A2D820688005F7D560680721490382
:107550008843296A084360606068297F0002000A46
:1075600009060843606011E0E2E02168FF20013075
:1075700081432160FFF736FA064604E0FFF732FA4E
:10758000801B022872D820688005F7D42878794EAD
:10759000000724D568690028306910D0012108430C
:1075A0003061FFF71FFA009005E0FFF71BFA009922
:1075B000401A02285AD830698007F6D50FE04008F3
:1075C00040003061FFF70EFA009005E0FFF70AFA7D
:1075D0000099401A022849D830698007F6D42878E3
:1075E000400766D500200290A06BC00006D4A06BB7
:1075F000012109070843A063012002905E48016849
:10760000C90511D40168821511430160FFF7EAF939
:10761000009005E0FFF7E6F90099401A642825D8A4
:1076200055480068C005F5D5FF20AA6801308242A0
:1076300003D131690143316111E001218902002A3E
:1076400007D005231B029A4203D132690A433261F3
:10765000EFE7326982433261306988433061A8685C
:10766000002810D0FFF7BEF9009008E05FE0FFF7B8
:10767000B9F901460098091A4048814257D8306943
:107680008005F4D50DE0FFF7ADF9009006E0FFF7B7
:10769000A9F90099411A3948814248D830698005D2
:1076A000F5D40298002804D0A06B01210907884373
:1076B000A063686A002866D00C2F3ED001263606EB
:1076C0000228206805D0B0432060FFF78BF90546FB
:1076D0002FE0B0432060FFF785F9074604E0FFF78D
:1076E00081F9C01B022822D820688001F7D4E96AFA
:1076F000A86AE2680843296BFD231B049A431143DF
:107700000843E060206830432060FFF76BF90546CE
:1077100004E0FFF767F9401B022808D820688001C1
:10772000F7D530E0FFF75EF9401B022801D90320AE
:10773000FEBD20688001F5D425E00128F8D0E0687E
:1077400001210904AA6A014091421AD10F2189043A
:10775000EA6A0140914214D1032189050840296B4E
:1077600088420DE0001002401EBB000828010020E6
:1077700020010020401002400070004088130000EB
:1077800001D00120FEBD0020FEBDF8B504000ED0E2
:10779000FF27606A0537002500280AD0256165614A
:1077A00026464036A562707C002807D00AE00120FA
:1077B000F8BD6068B842F3D0E561F1E73574204662
:1077C00000F03EF8022171742068026840239A4359
:1077D00002602123A26860689B021A40384010436F
:1077E000E3688A021340184323690B40217D184344
:1077F000C907C90F0843A169931019400843E169FB
:10780000382319400843216A802319400843A16A9C
:1078100093001940084321680860A0690421000C06
:107820000840616A102319400843216848602068B5
:10783000C1699143C1616565012070740020F8BD84
:1078400010B586B0044614216846FDF7B0FC104917
:107850002068884219D10F48416B8214114341635B
:10786000C16A01221143C162C06A00211040059023
:10787000E0200090022001900320039002910491E7
:10788000052069460007FEF7DDFF06B010BD0000C9
:107890000030014000100240094910B5401E8842E6
:1078A00001D9012010BD074C60610321081F02F0BF
:1078B00075FD0020A06107202061002010BD0000A0
:1078C000FFFFFF0000E000E0F0B502462032137E2B
:1078D000012B1ED0012515760223537606687468A5
:1078E000B3687027BC430F68274377600068AC0714
:1078F000A04205D0084CA04202D0084CA04204D1BE
:1079000080244968A343194381605576002010768E
:10791000F0BD0220F0BD000000080140001401404D
:1079200070B5050005D02C462034607E002802D0BA
:1079300006E0012070BD00202076284600F010F8F7
:1079400002206076291D286801F08AFF0120A077B7
:10795000A076E076207760776076002070BD00002A
:10796000006801218907884204D10348816B012204
:10797000114381637047000000100240F8B50546CE
:1079800004462035287E012817D001262E760220B5
:107990006876226890687727FF23B8431B029843D4
:1079A00090600A68502A31D00EDC202A4BD006DCC9
:1079B000002A48D0102A3AD145E00220F8BD302AEA
:1079C00041D0402A33D136E0602A27D0702A12D025
:1079D00001200003121A2AD0824228D1CB684A68BB
:1079E0008968206801F075FF206881680122920390
:1079F000114381601BE0CB684A688968206801F008
:107A000068FF216888683843886010E0CA68496860
:107A1000206801F0D8FF5021206806E0CA68496854
:107A2000206801F0E1FF6021206801F05DFF6E76C3
:107A300000202876F8BDCA684968206801F0C3FFB5
:107A400040212068F1E711462068EEE710B586B0C6
:107A5000044614216846FDF7AAFB01212068890726
:107A6000884212D10A49CA6A02200243CA62C96A1C
:107A70000190014005914102009100210291039182
:107A8000049069460348FEF7DDFE06B010BD000015
:107A90000010024000040050F8B5064604462036A7
:107AA000307E0D4601280BD0012008273076002AB1
:107AB00008D0042A16D0082A2AD00C2A4DD137E043
:107AC0000220F8BD206801F017FF20688169394362
:107AD0008161206881690422914381612068816904
:107AE000EA6812E0206801F01FFF20688169012226
:107AF000D2021143816120688269012189028A438F
:107B0000826120688169EA6812021143816124E080
:107B1000206801F022FF2068C1693943C1612068F3
:107B2000C16904229143C1612068C169EA6812E019
:107B3000206801F02DFF2068C1690122D2021143A3
:107B4000C1612068C269012189028A43C26120683B
:107B5000C169EA6812021143C16100203076F8BDA4
:107B600070B5050005D02C462034607E002802D078
:107B700006E0012070BD00202076284600F00FF8B6
:107B800002206076291D286801F06AFE0120A07796
:107B9000A076E076207760776076002070BD704731
:107BA00070B505462C4602202034002908D004294F
:107BB0000BD008290ED0627F012A10D0012070BDA1
:107BC000A27E012AFAD1A0760AE0E27E012AF5D14E
:107BD000E07605E0227F012AF0D1207700E060778F
:107BE0000122286801F068FE01222868920701211D
:107BF000904205D0074A904202D0074A904204D1F1
:107C000082685207520F062A02D002680A430260B5
:107C1000002070BD000801400014014070B504460A
:107C20000D460068002201F047FE2068016A0C4AF8
:107C3000114203D101684908490001600120203444
:107C4000002D06D0042D06D0082D06D06077002028
:107C500070BDA076FBE7E076F9E72077F7E7000054
:107C6000111100007047704770470000F8B50268B6
:107C70000446D06911689668814B05461D40202353
:107C8000002D6CD0F7077F4DFF0FBC460D402F43F2
:107C900079D02546C7078035002F06D0CF0504D5FB
:107CA000012717622A683A432A60820708D5F2073B
:107CB00006D0276802223A622A6804273A432A60DB
:107CC000420708D5F20706D02668042232622A68E5
:107CD000022632432A6002070AD50A461A4066463F
:107CE000324305D02668082232622E6816432E6081
:107CF000020508D54A0106D501222668D202326261
:107D00002A681A432A602A68002A30D0800606D5DD
:107D1000880604D5616E002901D02046884728686E
:107D200021688968490602D42821084225D02046C6
:107D300002F04FF820688168490619D58268402111
:107D40008A438260206F002812D04F498163206FE0
:107D5000FEF7DEFB00280AD0206F816B06E0850667
:107D600011D58D060FD5616E77E020468847F8BDA6
:107D70002046FFF779FFF8BD05E02046FFF774FFC6
:107D800000202860F7E7256E012D56D1C50654D591
:107D9000CD0652D510261662206881682546490610
:107DA000403500292ADA226F116849680904090C54
:107DB000E1D02F8B8F42DED969831168096889066B
:107DC00017D4016832019143016020688168490835
:107DD0004900816020688168402291438160E367A7
:107DE0000020206620680168B1430160206FFEF723
:107DF0006DFB288B698B401A81B21AE0298B6A8B44
:107E0000891A6A8B89B2002AB5D00029B3D00268DA
:107E1000FF252135AA43026020688268520852007B
:107E20008260E36700202066606620680268B243D3
:107E300002602046FFF716FF9DE7C50208D57502D0
:107E400006D50120000510622046FFF70CFF92E7DF
:107E5000050605D50D0603D5A16E002985D18AE753
:107E6000400688D5480686D5116820464024A1439F
:107E7000116083670021816600F043F97BE7000011
:107E80000F08000020010004F99C000810B5040050
:107E900003D0A06F002802D007E0012010BD002110
:107EA00074200155204600F027F82420A0672068A0
:107EB0000168490849000160204601F0DDFF012802
:107EC000ECD0606A002802D0204601F0F5FD206861
:107ED00041680922D20291434160206881682A22C8
:107EE00091438160206801680122114301602046AE
:107EF00001F048FE10BD0000F0B587B00646142121
:107F00006846FDF754F92C493068884251D12B4816
:107F1000416B0122920311434163C16A0122114363
:107F2000C162C06A00251040059003204002009005
:107F30000220032701A9A1C104200490052069465D
:107F40000007FEF77FFC1F4C1D48A560E56081C45B
:107F50008027E560A7602020256160610002A061A4
:107F60001848083CFEF74EFB002801D0FDF768FEDC
:107F70003467A662144C124821461438206003204E
:107F8000606010200831A1C16561A561E5612046EE
:107F90002562FEF737FB002801D0FDF751FEF4669D
:107FA000002201211B20A662FEF7A2FF1B20FEF784
:107FB00093FF07B0F0BD0000003801400010024000
:107FC00030000240E01500202816002070B5C36F75
:107FD000202B27D100290BD0002A09D00124836847
:107FE0002403A34206D10369002B03D1CB0701D0A0
:107FF000012070BD034660331C7D012C12D001248A
:108000001C7500230366084C0368A34207D05C6814
:10801000240204D51C680125AD062C431C6002F027
:108020002BF870BD022070BD0048004070477047BB
:10803000FFB50446806F83B017460D4620285ED1F9
:10804000002D0AD0002F08D0A168C001814207D1BD
:108050002069002804D1E80702D0012007B0F0BD54
:10806000204660300090007D012848D00098012112
:1080700001750020802108512120A067FEF7B2FC85
:10808000264640360190378277820120A16800039E
:10809000814202D12069002805D02F460025009991
:1080A0000020087511E00027F9E700228021204612
:1080B00002F028F8002815D1002F15D02168387853
:1080C00088627F1C708A401E7082708A019B002823
:1080D00006980090E9D100224021204602F012F8D3
:1080E000002808D00320B9E728882168C005C00D02
:1080F0008862AD1CE6E72020A0670020AEE70220E2
:10810000ACE7704701490248C160FDE70400FA0589
:1081100000ED00E030B585B014216846FDF747F862
:108120000D48408B012805D0022801D100F000FC49
:1081300005B030BD0122094D940221462846FEF7C4
:108140004AFC0021012002910391019000946946AC
:108150002846FEF777FBEBE7D40000200004005030
:1081600010B505242407002204212046FEF733FC25
:10817000002208212046FEF72EFC0A2002F0D5FE40
:10818000012204212046FEF726FC0A2002F0CDFE43
:10819000002204212046FEF71EFC10BD10B5052468
:1081A0002407002204212046FEF715FC01220821A5
:1081B0002046FEF710FC0A2002F0B7FE012204213F
:1081C0002046FEF708FC0A2002F0AFFE0022042140
:1081D0002046FEF700FC10BDF8B500240526074632
:1081E00025463607002204213046FEF7F4FB0A201C
:1081F00002F09BFE012204213046FEF7ECFB6006F4
:10820000040E08213046FEF7D9FB002801D0641C7B
:10821000E4B2052002F089FE6D1CEDB2082DE1D319
:10822000002F03D0FFF79CFF2046F8BDFFF7B6FFF5
:10823000FAE770B5052605463607002204213046C8
:10824000FEF7C9FB0024E80901D0012200E000226A
:1082500008213046FEF7BFFB6806050E0A2002F033
:1082600064FE012204213046FEF7B5FB0A2002F02D
:108270005CFE002204213046FEF7ADFB0A2002F02E
:1082800054FE641CE4B2082CDDD370BD10B5052487
:108290002407012208212046FEF79DFB012204212C
:1082A0002046FEF798FB002208212046FEF793FBAC
:1082B0000A2002F03AFE002204212046FEF78BFB42
:1082C00010BD10B505242407002204212046FEF726
:1082D00082FB002208212046FEF77DFB0A2002F0E7
:1082E00024FE012204212046FEF775FB012208210D
:1082F0002046FEF770FB0A2002F017FE10BD70B595
:1083000005252D070024012208212846FEF763FBDE
:10831000062002F00AFE012204212846FEF75BFB3C
:10832000062002F002FE07E0641CE4B2FA2C03D936
:10833000FFF7C7FF012070BD08212846FEF73EFB6E
:108340000028F1D1002204212846FEF744FB00203A
:1083500070BD0000F8B501F047FC01F081FC584801
:108360000068C069FDF75CFD564C5749A082898FB3
:10837000564E0025002931D0A26A730354499A420F
:1083800002DB02220A7000E00D700A7801218902E6
:10839000002A05D0012A0ED0022A10D0032A1DD1AE
:1083A000608B01282BD0022818D14548082140387D
:1083B000FFF734FC12E0FF22F5329042F0D2608BDE
:1083C00001281AD0022804D008E03046FEF703FB4B
:1083D00004E03B4808214038FFF7E2FB0121C902D5
:1083E0003046FEF7EBFA0127FF0300282AD0394870
:1083F0000560E079002804D007E00022E5E70122CB
:10840000E3E70120E07101F0DFFE2078632806D960
:10841000002208213046FEF7DEFA012205E00122A3
:1084200008213046FEF7D7FA00220520394600071A
:10843000FEF7D1FA244C284E4034A08C274F012857
:1084400003D01CE0E5710022EAE725486946088070
:1084500072B680212348FDF70BFC002804D00222CD
:1084600069462048FDF7A8FC62B61FA001F04AFF4C
:10847000A58403F0D5FA642002F050FDFE60608C04
:10848000012808D110486584058003F0C9FA6420EA
:1084900002F044FDFE60208C012806D1258403F003
:1084A000BFFA642002F03AFDFE600748124A0188D4
:1084B000914202D1C088002800D1FE60F8BD0000C2
:1084C0005C150020D40000205C0D0020000400504A
:1084D00069000020180100200400FA0500ED00E00A
:1084E000AAAA0000384A0008BDF8C8EBC9FDBCB60E
:1084F000C4A3CABD0D0A0000AA55000008B5372163
:10850000202000F06EF80321212000F06AF84021BD
:10851000222000F066F80821232000F062F8AA214A
:10852000302000F05EF80A48008FC1B2322000F01F
:1085300058F80221332000F054F85F21202000F089
:1085400050F8684600F006F80A2002F0EEFC08BD7C
:108550005C0D002010B501460F2000F021F8002826
:1085600000D0012010BD10B50446FFF78FFE322069
:10857000FFF75FFEFFF7C3FEE0B2FFF75AFEFFF71B
:10858000BEFEFFF783FE3320FFF753FEFFF7B7FE73
:108590000020FFF721FE0446FFF793FE204610BDA2
:1085A00010B50C46FFF7DFFF2070012010BD70B53D
:1085B0000D460446FFF76AFE3220FFF73AFEFFF74A
:1085C0009EFEE0B2FFF735FEFFF799FE2846FFF763
:1085D00030FEFFF794FEFFF774FE0A2002F0A5FCC0
:1085E00070BD10B5FFF7E3FF012010BD10B50248C4
:1085F000FEF731FB10BD000094140020FEB50446C8
:10860000002772B6334A01688B1804D13248C76814
:1086100003208004074088680190C868009048697A
:108620008E69002B08D12C4940398B6ACD042B432D
:108630008B628B6AAB438B62014631433CD0254948
:108640002368CB4205D12449CA6803239B049A437B
:10865000CA6025462035002810D021680A69012308
:108660001A430A61216848610821204600F036F863
:10867000032800D1A873216808204860002E10D07C
:10868000206801690122114301612068866110217F
:10869000204600F023F8032800D1A8732168102099
:1086A00048600C482168C14206D10B48C1680322CA
:1086B000920491433943C160206801694908490027
:1086C000016121680198886021680098C86062B6DD
:1086D000FEBD00000084FFBF4010024070B506469A
:1086E0000B480D46002409490068FCF701FD7D2177
:1086F000C90048433168401E00D103240B682A4654
:108700009A4301D00028F6D1204670BD204E0000CB
:10871000280100201CB5002116480091144A01913F
:108720000260C163120542608160072282630122F8
:1087300002610246C16020321170FF235170C233C2
:10874000436281621173016381610422416342616A
:10875000C161FDF721FD0848009080130190694632
:108760000448FDF7C9FC00210248FDF76FFC1CBD61
:1087700000240140381400200200000408B5084815
:10878000016B012211430163006B01211040009035
:1087900000220A20FEF7ACFB0A20FEF79DFB08BD75
:1087A00000100240F0B587B014216846FCF7FFFCCA
:1087B0004748C26A04210A43C262C26A0A4005925B
:1087C000C16A80263143C162C16A31400591C16AE4
:1087D00001242143C162C16A21400591C16A022579
:1087E0002943C162C06A22462840059005201C2109
:1087F0000007FEF7F0F8012236493748FEF7EBF89C
:10880000002236493448FEF7E6F89121052000227F
:1088100009020007FEF7DFF8314801900027052024
:108820006946029700940007FEF70CF80C200090B0
:10883000112001900320039005200297694600074C
:10884000FEF700F810206A46039591C2052069469C
:108850000007FDF7F7FF1120019002976946039783
:1088600000941D48FDF7EEFF1E48019069460095F3
:1088700002941948FDF7E6FFE0020090694601976F
:1088800002951548FDF7DEFF1748694691C1694614
:1088900011480397FDF7D6FF91200002694691C168
:1088A0000520694600070397FDF7CCFF69460A4893
:1088B000019700960294FDF7C5FF002201210520D3
:1088C000FEF716FB0520FEF707FB07B0F0BD000022
:1088D00000100240010200000004005008300000B7
:1088E00000001110000021100832000010B50F4CDC
:1088F0000D482060FF20053060600020A060E0602F
:1089000020616061E0610121206249026062A16131
:10891000A0620720E0622046FEF737FF206801686A
:1089200040221143016010BD00300140C4140020FA
:1089300010B58AB000240494059406940794089412
:108940000121184809940094019402948907039422
:108950000160092184604160046113494461C16080
:10896000FEF7DEFF01200003049004A90D48FFF785
:1089700005F80C48FFF7F4F8089408A90948099489
:10898000FEF7A2FF602000900848019002940822A0
:10899000694603940348FFF77FF80248FFF756F84B
:1089A0000AB010BD1C1500209304000057020000FF
:1089B00000B585B014216846FCF7F9FB0E480D4957
:1089C0000160E1214902416000218160C1600161D3
:1089D00081610C22C1614261016230214162012149
:1089E000090381634900C163FFF750FA01F0E6FB18
:1089F00005B000BD003801405C1500207047000044
:108A0000F0B587B00A2002F079FD7D20C00002F0A9
:108A10008FFDFB4C0020A070FA49A164617B0C29FA
:108A200001D30B2161730025F748E570F74E0078FC
:108A30003071F749A079097840000843E17C89004A
:108A40000843F071A06AF070401CA0626079314662
:108A5000B0744200B4310846A138FCF78FFB062001
:108A60007072EC4831460078B072A07E30731339D2
:108A7000207F0875607F48756079002240001331BF
:108A8000153002F025FE607900214000153002F01B
:108A900031FE022002F082FDF571E573A572012618
:108AA0002673E572DC48FEF7B1F920840746E570CD
:108AB0006079FCF7E3FDD94AD94BFCF7D9FC02F009
:108AC000C9F90022B307FCF721FCFCF71DFE0006E4
:108AD000C10CC81980B2F1036084884201D3401AE6
:108AE0006084D04860632079401C2071CA48FEF73A
:108AF0008DF9E083C5480C3005464235403003907F
:108B0000B5E1C548FEF782F9E083C74F0BE0C248E4
:108B1000FEF77CF980B2E083618C884203D3C34ABC
:108B20008918884206D300210F2002F067FC3842E2
:108B3000E062ECD0E06A411C21D040047ED5812265
:108B4000D20100210F2002F098FD7D20C00002F02C
:108B5000EFFC002002F0A1FC0021102002F04EFCEE
:108B60004106AA48490E274600225030616402F0AF
:108B70007BFCA6485030417A0729C1D101E001F0C1
:108B80002FFC0222AA49401DFCF71CFB0028B7D18C
:108B900002F001FE7965386502F0EAFDF965B86515
:108BA000F8786946401CF87098484D3002790A7090
:108BB0004079487008880490B98B88427ED19D4FD7
:108BC000288A38800398808A20839348FEF71EF90C
:108BD000E08302F025FBFF22A16D5204E06D00232B
:108BE000891858410206080A1043009040084000C6
:108BF000010E0002616620668448636D0A30226DB2
:108C000002F09EFD6079E36D81008048A26D081836
:108C1000163002F095FD7D48636E1230226E02F030
:108C20008FFD7A4808214172A07C002816D0774831
:108C300002227F495530FCF7C5FA00E00AE100281E
:108C40000CD17248E673C671606C70491638C2B2B6
:108C5000663108462274EA30FCF790FA6079002207
:108C600080006A491C3002F033FD607900218000E9
:108C70001C3002F03FFD009802F039FC012002F0A8
:108C80008DFC207202216C48FDF798FE00287DD0F3
:108C900000215F4801705A48A9890186EA89428605
:108CA000206B606359485030C37C1807000F0328BD
:108CB00000D060741809A074002000E06FE02071FB
:108CC0004F4BA6729986DA86E672218B5B4AFF319A
:108CD000C33189B2218391420BD952428918218331
:108CE00039887D22491C89B2D2003980914200D353
:108CF00038803D887D20C000218B68434018A063E8
:108D000006904F48302107784E48A77300884843A3
:108D1000FCF799FC019028460A214843FCF793FC94
:108D20000199FCF7B5FA7F21C905FCF758FAFCF761
:108D3000B3FC80B242497F1E0880B84200D1E6727F
:108D4000A5841420205EFCF785FC06460F46E08BC8
:108D5000FCF794FC3C4A3D4BFCF78AFB0546059129
:108D60000698FCF777FC2A46059BFCF773FB324616
:108D70003B46FCF7CBFAFCF7A3FCE063608B00F00A
:108D8000A7FC207A002803D07AE0FFE7012180E7E2
:108D900000210F2002F032FB0006F9D570E0FDF74C
:108DA00027F82B4A032111541549AA890A86EA8912
:108DB0004A86274980006039421803990190098B3F
:108DC0001180234A396B303A11501049FB6D40181D
:108DD0001630BA6D02F0B4FCB96C386B884200DA18
:108DE000B8641B4A0199603A515881423FDD00291D
:108DF0003DD000283BDD0498B8830220387036E06F
:108E0000580000203F420F00D4000020D011002065
:108E100014010020E400002094140020B81E85EB0B
:108E200051B8CE3FA086010000D02724983A000018
:108E3000F80000201001002000040050E7030000AB
:108E4000F0000020F4000020F853E3A59B843E408E
:108E5000141300203A4600210F2002F00EFC607926
:108E6000E178401C814202D0002002F016FBE18B29
:108E7000608C814200D244E6274A80188142FAD8A9
:108E800002F0CEF9254A00210F2002F0F6FB2079EE
:108E9000002807D022490A2209885143814201D281
:108EA00000202070E07B00281BD01E490B784878FA
:108EB0008A78022B15D1102804D11B4D2B685B003A
:108EC0001B0E0AD0194BC91C1818FCF757F902F0F1
:108ED000A7FD642002F022F851E6C878FCF7B3FB46
:108EE0002860104D00209C3D2E462178627918366E
:108EF00007E04300EF5AF35A9F4200D00221401C82
:108F0000C0B29042F5D3054A2170803200210F2073
:108F100002F0B3FB07B0F0BD983A000000D0272460
:108F2000E400002020130020FC0000205C0D002045
:108F300070470000F0B58DB0B44801900020C043E8
:108F40000A9000260A2002F0D9FA7D20C00002F023
:108F5000EFFA0020AE4C0546A070AE4FAE480B9025
:108F6000AD480022C23885730146142002F0B0FBE0
:108F70000021142002F0BEFB022002F00FFB0021B2
:108F80000F2002F03BFA3842E062F8D0E06A411C60
:108F900018D040047ED58122D20100210F2002F09A
:108FA0006CFB0021102002F029FA41069A48490E74
:108FB0000022801C02F058FA9748801C417A02294E
:108FC00002D007E101F00CFA934802229349C01D38
:108FD000FCF7F8F80028F4D102F0DDFB61652065AC
:108FE00002F0C6FBE165A065002E22D10B988C49EA
:108FF000008A088088480126801E808A208389484C
:10900000FDF704FFE083208B8749FF30C33080B237
:10901000208388420DD9494240188149208308881D
:10902000814A401C80B20B320880904201D300205C
:1090300008800B9968468A890280C98941807649EF
:109040000422C91C0846A238FCF798F8FF22A16D3B
:109050005204E06D0023891858410006090A0143B3
:109060000846029102F043FA029948084000010EB6
:109070000002616620666848636D9638226D02F0D2
:109080005FFB6548E36D9238A26D02F059FB6248C0
:109090008E3800E0A0E0636E226E02F051FB5E4964
:1090A0000022A0393C2002F013FB00213C2002F0FA
:1090B00021FB012002F072FA2072A0780121401CED
:1090C000A0700520C9030007FCF7A6FE54487D22C6
:1090D0000088D200014602905043228B0A39801842
:1090E000A0630C9051480078A073049008B2E0840B
:1090F000002803DA7D21C9004018E0844C48302163
:1091000000884843FCF79FFA05902620205EFCF774
:109110008FFA0599FCF7BCF87F21C905FCF75FF8C9
:10912000FCF7BAFA414980B208800499491E884286
:1091300001D10120E0720298A0841420205EFCF787
:1091400089FA05910690E08BFCF798FA394A3A4B78
:10915000FCF78EF9079104900C98FCF77BFA079BBB
:10916000049AFCF777F9059B069AFCF7CFF8FCF711
:10917000A7FAE063608B00F0ABFA00990198814296
:1091800010DA00290ED024490422C91C0AA8FBF7D2
:10919000F5FF0220207029480A21007848436072B8
:1091A00000980190207A002805D100210F2002F0BC
:1091B00025F90006F9D5802200210F2002F05DFA82
:1091C00000206D1CEDB26070032D00D2C8E6002EA9
:1091D00008D017E00120F4E7194A00210F2002F01F
:1091E0004CFAF7E7618B1748002902D002889142B8
:1091F00001D90188618388B21349401E0988484318
:10920000124908800A98A0830DB0F0BD3F420F00BC
:109210005800002000D027241E120020F800002053
:109220001001002094140020E7030000F00000204B
:10923000F4000020F853E3A59B843E40E4000020A6
:1092400000902724E0000020DE000020DC00002049
:10925000F8B53A493848086002F084FB384800F015
:10926000F7F9384CE0823648801C00F0F1F9208391
:109270003348001D00F0ECF96083852132488900F5
:109280004180014640310979304F0906090E61706D
:1092900003D0C188002908D009E0C7800121C18717
:1092A0000A2141870021818701E06421C180018F6B
:1092B0000A2901D902210187C18E3C2901D93C210B
:1092C000C186234A89B21170C18F6171818FA171EA
:1092D000817AE1708588052165626181C6883046A2
:1092E000FBF706FFA08101462846FBF701FF880037
:1092F000081885B2154825816843FCF7BFF9154A5F
:10930000154BFCF71DF9FCF7FFF9E081658231464A
:109310003846FBF7EDFE20820146C820FBF7E8FE49
:1093200020840120A083FCF77BFDA082E2890B4909
:109330000B48FDF76FFDF8BDF5A1000850000020B7
:10934000004F0008D40000205C0D0020E80300005E
:1093500000000020F853E3A59B843E40FF7F0000FF
:1093600094140020F0B5954D85B001202880944FCD
:10937000C820944C3880E079401CE071C00706D0CA
:10938000608B411E6183022801D2C8206083608BFC
:1093900000F09EF90A2002F0B1F87D20C00002F032
:1093A000C7F802218848FDF709FB002838D00020C3
:1093B000864980000978874E490008438449097826
:1093C0000843B072102070728348C1887D20C000AD
:1093D000FBF78EFE707381487F490078B07330468A
:1093E0000B308A780270C9784170411C7A4820306D
:1093F000027ECA70407E087177482230027E4A7130
:10940000407E887100220C39152002F061F900219C
:10941000152002F06FF9022002F0C0F8704E03E050
:109420000120C5E7FEF796FF00210F2001F0E6FFBF
:109430003042E062F6D0E06A411C7DD040047CD529
:109440008122D20100210F2002F017F90021102003
:1094500001F0D4FF41065F48490E0022503061649C
:1094600002F002F85B4E5036707A112865D1022264
:109470005C49701DFBF7A6FE00285ED1F01E027944
:1094800069460A7040794870B17A2980C820FBF794
:109490002FFE3880307B6083534DB01E008A2880B9
:1094A000301F808A20835148FDF7B0FC80B2E083F2
:1094B0000390208B4E49FF30C33080B22083884216
:1094C0000CD949424018208328884949401C80B261
:1094D0000B312880884201D3002028802D887D20F0
:1094E000C000218B68434018A06301904148067872
:1094F00028460A3800B2A673E084002803DA7D21EA
:10950000C9004018E084388830214843FCF79BF8B4
:1095100007462620205EFCF78BF83946FBF7B8FE9D
:109520007F21C905FBF75BFEFCF7B6F880B2314935
:10953000761E0880B04201E03EE03BE001D1012010
:10954000E072A5841420205EFCF784F802900F4698
:109550000398FCF793F8284A284BFBF789FF054648
:109560000E460198FCF776F82A463346FBF772FF61
:109570003B46029AFBF7CAFEFCF7A2F8E063684696
:109580000088A083134813495030807C6331607198
:10959000420008460D465130FBF7F0FD6079294640
:1095A00042000C48CC30FBF7E9FD608BFF2801D06E
:1095B0000320207005B0F0BD00F012FFE400002091
:1095C000F40000205800002000040050D9000020C2
:1095D000DA000020D01100205C0D002000000020E7
:1095E00000D02724F800002010010020941400204F
:1095F000E7030000F0000020F853E3A59B843E4001
:1096000070B586B014216846FBF7D1FD01250F4ED9
:10961000ED03002229463046FDF7DDF90120002444
:10962000019002946946009503943046FDF70AF9CB
:109630000320019002946946009503943046FDF79B
:1096400001F9022001F06AFC06B070BD0004005070
:109650000088704770470000F8B5044600206A464D
:109660001080194D55222A70AA226A700322AA700E
:10967000661DEE702A716971144A49008918AC712F
:109680002246E81DFBF77AFD002007E029186A460C
:109690008978128889186A461180401CB042F5DB2F
:1096A000611DA81CFCF712FA0146684601802919C1
:1096B0000078C8716846407808722146093102482E
:1096C00000F0A8FBF8BD0000D41300205C0D0020C2
:1096D00010B51B4C228A01E0891AA183A18B91420B
:1096E000FAD2228C8BB253431B18E383132902D185
:1096F0004A431018E083E08B3021484364216430F2
:109700004843104960630968401A4B210901401819
:109710002063FBF79FFF0C4A0C4BFBF711FFFBF795
:10972000CFFF0B49E062884202DD4A428018E062C6
:10973000002801DA4018E06206490968486110BD56
:10974000D400002094000020F853E3A59B843E4001
:10975000FF7F000094140020034A1168382389B267
:1097600099430143116070470030014010B5FDF787
:109770003FF910BD10B59AB034216846FBF717FDCC
:1097800014210DA8FBF713FD1C2112A8FBF70FFDF8
:109790001B4801680324E402A143C2148918016034
:1097A000FDF7B2FB17480169A14301610620009053
:1097B000FF2001300290012003901020049002202D
:1097C000099040040B90000100240C900A94684614
:1097D000FDF7C8FD0F200D9003200E900F941094FC
:1097E000012111940DA8FDF793FC81201290032014
:1097F00080041890149412A8FDF7D8FB1AB010BD7D
:10980000007000404010024010480168821511436A
:109810000160C1680E4A1140C16001680D4A1140E3
:109820000160816849084900816001680122920451
:1098300091430160C168FD2212049143C16000217F
:10984000016106490448886070470000001002402A
:109850000C40FF88F6FFF6FE0050000800ED00E027
:1098600070B5026801239B07114C124D984203D03A
:10987000A04201D0A84203D17026B2434E683243C1
:10988000984203D0A04201D0A84204D103231B0276
:109890009A43CB681A4380239A430B691A430260A8
:1098A0008A68C262096881620121416170BD00005D
:1098B000000801400014014010B5CB06DB0E012169
:1098C000046A99408C430462016A9A401143016220
:1098D00010BD30B58468FF252D021B021343AC4335
:1098E0000B432343836030BD826870239A430A434D
:1098F00007210A438260704730B5026A520852005D
:109900000262026A456883697024A3439C080B685D
:10991000A40023430224A2438C684560144383615E
:1099200049684163046230BD30B5026A10239A432E
:109930000262036A4568826973242402A2430C68A8
:1099400024021443202293438A68456012011A437B
:10995000846149688163026230BD30B5026AFF23C9
:1099600001339A430262026A4568C3697024A343C3
:109970009C080B68A400234301246402A2438C6862
:10998000456024021443C3614968C163046230BD69
:1099900030B5026A01231B039A430262036A4568D9
:1099A000C26973242402A2430C68240214430122D6
:1099B000520393438A68456012031A43C46149689D
:1099C0000164026230BD30B5036A046A6408640051
:1099D00004628469F025AC43120122430A24A343A4
:1099E0000B438261036230BD30B5036A1024A34388
:1099F00003628469036A0F252D031203AC432243DB
:109A0000A024A343090119438261016230BD000013
:109A100070B5102405252D07AC62AF20800001F041
:109A200084FAAC6101F0FEFC214C224EE06402E0BD
:109A300001F0F8FCE064B042FAD120780126F60388
:109A4000002806D001280CD0022817D003282BD1DB
:109A500028E0012231462846FCF7BDFFFFF782FCD3
:109A600006E0012231462846FCF7B5FFFFF762FA0F
:109A7000002231462846FCF7AEFF15E0607A01224D
:109A8000401E607231462846FCF7A5FFFCF7E4F95A
:109A9000002231462846FCF79EFF607A002803D159
:109AA000207001E0FEF7ACFF01F0A2FB70BD0000EA
:109AB000580000203001CADE10B5818CC90707D0DC
:109AC00001684A6801235B049A43836A1A434A6027
:109AD000818C890707D501684A6801231B049A43D2
:109AE000C36A1A434A60818C490707D501684A68EE
:109AF00001239B049A43036B1A434A60818C090734
:109B000007D501684A680123DB039A43436B1A4374
:109B10004A60818CC90607D50268916801231B033E
:109B20009943836B19439160818C890607D501683D
:109B30008A6801235B039A43C36B1A438A60818C52
:109B4000490612D503685A6801210905046C8A4345
:109B500022435A60026C8A4207D10268516803238B
:109B60005B059943436C19435160818C090607D505
:109B700001684A680123DB04806C9A4302434A600F
:109B800010BD0000F8B50446002680300660FCF7E2
:109B900029FF054620680068124F000709D50121FA
:109BA0002B46002249052046009700F0ABFA00281A
:109BB0000DD12068006840070BD501212B460022FB
:109BC00089052046009700F09DFA002801D0032067
:109BD000F8BD2020A067E067266660342675002067
:109BE000F8BD0000FFFFFF01F8B5184CC826E0786B
:109BF000002829D16079002826D101206071144DF8
:109C0000686B002700281ED0686BC821081A15E071
:109C10001048E168405C616988470F480A21008864
:109C200048430E490880E068401CE060E068C828AE
:109C300000DBE760696BC820401A761EE16881424C
:109C400001D0002EE4DC6771F8BD00003C0000206C
:109C500000000240940C0020E4000020F6000020E8
:109C600070B5224CE07800283FD1207900283CD103
:109C7000012020711E4EF16900250906002933DA02
:109C80002156625791420AD1F06940062CD5A0793D
:109C9000002829D0A5712089401C208124E0A179C9
:109CA000002903D1A0710A2001F03FF900202056BD
:109CB000CC2148430F494218206912181279B26228
:109CC000401C00222061A256CC235A43895881426D
:109CD0000ADC25612078401C207020780E2800D1F5
:109CE0002570A078401CA070257170BD3C0000203C
:109CF000003801406C01002010B5806A0022014646
:109D000040314A834A82FDF7AFFF10BD70B5846AC7
:109D1000A06FE56F2168896800260906002906DA28
:109D2000212804D152200653204600F06BF8206809
:109D30008068400606D5222D04D15A2006532046BD
:109D400000F047F82046803001681022114301607E
:109D50002046FDF789FF70BD10B501460968806A8D
:109D6000096889061CD400225A210A5201680A682F
:109D7000FF2301339A430A6001688A68520852003F
:109D80008A6001688A6840239A438A602021C167FB
:109D9000016E012904D101680A6810239A430A6000
:109DA000016E012902D0FEF741F910BD5821095A70
:109DB000FDF758FF10BD10B5806A016E012902D071
:109DC000FEF735F910BD5821095A4908FDF74AFF39
:109DD00010BD01680A68FF2321339A430A600168B5
:109DE0008A68520852008A60016E012904D1016814
:109DF0000A6810239A430A602021C1670021016686
:109E00004166704701680A68C0239A430A602021AE
:109E10008167704770B5164CE278002A0CD1227920
:109E2000002A09D10122E2700025C82903DC0222A0
:109E3000A256002A01DCE57070BD0123E356CC2256
:109E400053430C4AD1500123E356CC2673439B184D
:109E50000A460146181DFBF791F96078401C6070B6
:109E600060780E2800D16570A078401EA070E2E7EF
:109E70003C0000206C010020F8B5044601688068B1
:109E80002369E66918436369002533431843724A1E
:109E90000B68724E334003430B602168486803230C
:109EA0001B039843E368184348602168A069914206
:109EB00001D0236A18438B680B263602B343034351
:109EC0008B606749236867488B420CD1C068800764
:109ED000800F06D0012839D0022835D0032821D19F
:109EE0001EE001271FE060498B420AD1C0680C21A7
:109EF000084027D0042829D0082825D00C2811D1C3
:109F00000EE093420ED1C16803208002014019D0B7
:109F100001208002091A19D0091A15D0814201D1F5
:109F2000082700E010274F495048403986009342E7
:109F300032D1002F0CD0022F0DD0042F10D0082FBB
:109F40007FD126E00027EEE70227ECE70427EAE7C7
:109F5000FDF7ACF906E00968C90605D4304603E010
:109F6000FDF7C4F9002872D062685100511881428F
:109F700067D81103814264D3010E06025008002302
:109F800030185941FBF7CAF803210902411A384A2F
:109F900055E00120C003E7E70122E369D2039342C1
:109FA0002BD13B0000F0EDF90906090C4D114D4D88
:109FB0004D274D00FDF77AF909E0FDF787F906E036
:109FC0000968C90605D4304603E0FDF78FF900287B
:109FD0003DD0616840004A088018FBF789F880B2DC
:109FE0000146244A103991422BD8511C01400007E8
:109FF000400F084329E01046EBE73B0000F0C1F9B1
:10A000000906090C2112212121232100FDF74EF917
:10A010000AE0FDF75BF907E00968C90606D4304697
:10A0200004E00EE0FDF762F9002810D061684A08EC
:10A030001018FBF75DF880B201460E4A10399142C4
:10A0400003D9012503E01046F0E72168C86000202D
:10A050006066A0662846F8BD00480040F369FFEF3F
:10A0600000380140401002400044004000093D001B
:10A07000FFFC0F00EFFF0000F8B5044641654030DB
:10A0800000262746028380373E602220E06725466F
:10A09000206F603500281CD01749C162216F174816
:10A0A0000863216F16484863206F8663236F606DD5
:10A0B0009C4613462168024660462431FCF7EAFAC2
:10A0C000002806D0102038602E752020A0670120BF
:10A0D000F8BD2E7520680168FF220132114301602E
:10A0E00020688168012211438160206881684022D4
:10A0F000114381600020F8BD599D0008B79D0008FC
:10A100000D9D0008FFB581B005460F460446603539
:10A110000A9E39E0701C37D0FCF764FC0499401AA1
:10A12000B04222D8002E20D02068016849072BD5E4
:10A13000C069C043000527D401202168C00208621D
:10A1400020680168FF22A132914301602068816884
:10A150004908490081602020A067E06780342060C2
:10A1600000202875032005B0F0BD20680168FF229B
:10A17000A1329143016020688168490849008160EB
:10A180002020A067E067EBE72068C1693846884374
:10A1900005D0002103988142BCD00020E3E70121D3
:10A1A000F8E7000010B50449102009680862024869
:10A1B000FDF75CFD10BD00005C15002001490D207D
:10A1C000887070473C00002010B507480A22018AB9
:10A1D00051434184FEF7D2FAFEF7EAFBC822034955
:10A1E0000348FDF7F3FE10BDD4000020940C0020BE
:10A1F0005C150020F8B53E4C002321783D4A1D46F1
:10A20000082910D0072947D0062950D0052952D057
:10A21000042953D0032954D0002956D0012958D0FD
:10A2200002295AD05BE0A17800264A1F04E0314F92
:10A23000BF5DFB189BB2761C9642F8DB66792779E6
:10A240009A195118E3786278C9188918C919401801
:10A25000C0430006000E1AD1012E14D0022E16D1D2
:10A2600025482449C018FAF789FF01F0D9FB64207A
:10A2700000F054FEBFF34F8F21492048C860BFF360
:10A280004F8F00BFFDE759081046FFF7E5F925702D
:10A29000E570A570A571F8BDA1795054491CC8B2EC
:10A2A000A071A178491F8842F5D1082001E06070B3
:10A2B00007202070F8BDE0700620FAE760710520E5
:10A2C000F7E7A070E5700420F3E7552807D10120D7
:10A2D000EFE7AA2803D10220EBE7032803D025707B
:10A2E000E570A570F8BD032020702071F8BD000056
:10A2F000CB000020701300205C0D00200400FA0544
:10A3000000ED00E00FB410B503A9044B044A029815
:10A3100000F004FA10BC08BC04B0184759B7000894
:10A320002C0100202021020C01D010211046020A2D
:10A3300001D010460839020901D01046091F8208D1
:10A3400001D01046891E420801D0881E7047081AA5
:10A350007047F8B5040C8BB2264682B25E430D0CF2
:10A360001046370C584336048019002179411646AF
:10A370006E43370C36048019794126466E4389199D
:10A38000F8BD30B47446641E2578641CAB4200D21C
:10A390001D46635D5B00E31830BC18478307FF224E
:10A3A000DB0E9A408907090E9940002808DB8308D4
:10A3B00009489B001B1818689043084318607047B1
:10A3C0000007000F0838830804489B001B18D86951
:10A3D00090430843D861704700E400E000ED00E0DE
:10A3E000BFF34F8F04490348C860BFF34F8F00BFCE
:10A3F000FDE700000400FA0500ED00E002E008C8F7
:10A40000121F08C1002AFAD170477047002001E0EE
:10A4100001C1121F002AFBD1704708B50021684610
:10A4200001706B46012202212C2001F035F9022136
:10A43000684601706B4601222C2001F02DF908BD01
:10A4400038B504466D20694608706B4601220749FD
:10A450002E2001F021F90649002C01D0054A00E028
:10A46000054A2E2001F0FEF838BD00000608000065
:10A4700006180000070600000716000038B504465D
:10A480006B4602220021362000F0D2FFB3212300C8
:10A49000FFF777FF0E0F08153A3A3A3A1C273A3A77
:10A4A0002F34483A0021684601704078410849003D
:10A4B00014E06946087880088000401C04E0694682
:10A4C000087880088000801C08701DE068460278CB
:10A4D0000A4048320270417880200143684641704A
:10A4E00012E0684602780A40027040784106490E40
:10A4F000F4E7694648780221084303E06946487852
:10A50000FD210840694648706B4601220021362033
:10A5100001F0C2F8012200AB11463620013301F0F0
:10A52000BBF838BD69460878CF210840694620301D
:10A53000CAE708B5032168464170012101706B46E6
:10A5400002220021362001F0A7F80122D2030621C1
:10A550002D2001F087F8012000F0E0FC0120FFF73A
:10A560008DFF08BD08B5020A69464A7008706B463F
:10A57000022204212D2001F08FF803206946087083
:10A580006B46012206212D2001F086F80020694645
:10A5900008706B46012206212D2001F07DF80A216A
:10A5A0002D2000F02BFF08BDF0B51FB486B0099830
:10A5B000089A030D0021024314D05148514A18183B
:10A5C000504305141198012810981AD0281A401CDD
:10A5D00000264D4F4D49009601910490002812DA53
:10A5E000444211E01198012449A3012801D1109897
:10A5F000C1430698119A84600360C26041600BB049
:10A60000F0BD4042E4E70446210500203F4A001C1B
:10A6100051410391029012E0E00707D032463B46D9
:10A6200001990098FAF724FF0191009032463B46C9
:10A6300010461946FAF71CFF06460F466410002C18
:10A64000EAD10498039B0028029A0999089806DA2F
:10A65000FAF70EFF019B009AFAF70AFF05E0FAF7F6
:10A660006FFF019B009AFAF76BFF04460E4600222B
:10A67000284BFBF77BF803D80020C043014607E0D6
:10A680000022254B20463146FAF740FEFBF77CF9C5
:10A69000102409E0002C0ADB0A220023FAF73EFD11
:10A6A000079B30321A55641E02460A43F2D111222A
:10A6B000641C079B121B1C19119B012B03D0012347
:10A6C00008430ED10AE0084304D011201090002066
:10A6D000119077E71098151A6D1E0BE010988242C2
:10A6E00002DD00236D1C03E0824201DA00236D1EAF
:10A6F000002BEED0069811998260C16030C07EE7D1
:10A7000001FCFFFF104D0000000014400000F03F6E
:10A71000300000000000F0430000E03FFFB597B0BC
:10A720000646002518E2252877D100242746FD4952
:10A73000049400E00443761C32780120203A9040D3
:10A740000842F7D130782A280ED00222307801460C
:10A750003039092916D804990A2359433039401849
:10A760001443761C0490F1E7189802C804911890DD
:10A77000002904DA012040030443484204900220E7
:10A780000443761C30782E2814D1042004437078BA
:10A79000761C2A2809D11898761C80C8189009E0E0
:10A7A0000A214F43303FC719761C307801463039B3
:10A7B0000929F5D930786C2810D006DC4C281AD03D
:10A7C00068280ED06A2817D104E0742813D07A289C
:10A7D00012D110E00120400504430CE001210905DD
:10A7E00001E0032109050C437178814203D1012066
:10A7F00000052418761C761C3078119066280BD042
:10A8000013DC58287DD009DC00287BD04528F6D001
:10A810004628F4D047281AD1A5E118E0632835D09E
:10A82000642870D0652812D19DE170286CD008DCB6
:10A830006728F1D069287BD06E280DD06F2806D10B
:10A84000BAE073282ED0752871D0782859D01A9A7A
:10A85000199990476D1C7EE16002400F022809D0D3
:10A8600003280DD00428189801680DD00D60001D34
:10A87000189070E11898EA1701680D604A60F6E7D1
:10A88000189801680D80F2E70D70F0E718986A4695
:10A8900001781172001D18900020507202A80090DB
:10A8A000012005E0189802C8189000200091C043CC
:10A8B00061070DD5002101E00199491C0191B942C0
:10A8C00012DA8142F8DB009A515C0029F4D10BE0E6
:10A8D000002101E00199491C01918142FADB019AB2
:10A8E0000099895C0029F5D1019904981A9B471AAF
:10A8F00021463846199A00F097FA019940194518EF
:10A900000BE04FE02CE113E04EE000980099007856
:10A91000491C00911A9A199990470198401E01907C
:10A92000401CF2D1214638461A9B199A10E137E0B3
:10A930000A200021009001916002410F022907D0F6
:10A94000189A01CA1892C2179446032908D00AE03F
:10A950001898C01DC108C90005C91891944607E0A0
:10A9600000B2C2179446042902D140B2C1178C46E6
:10A9700000226146944506DA0A4600214042914190
:10A980008C462D2102E0210504D52B216A46117346
:10A99000012103E0E10701D02021F7E7029155E012
:10A9A0000A200AE0102008E0102000900021042076
:10A9B00004430191082703E0082000210191009041
:10A9C0006002410F022907D0189A01CA189200228A
:10A9D0009446032908D008E01898C01DC108C90092
:10A9E00005C91891944603E080B2042900D1C0B291
:10A9F00000210291210729D51199702906D0009ACA
:10AA00001021019B4A401A4305D00EE040216A46BE
:10AA10001173012108E06146014306D030216A46E6
:10AA200011731199517302210291009A0821019B1F
:10AA30004A401A430AD16146014301D1610705D555
:10AA400030216A46117301217F1E02911199582904
:10AA500004D035A10E910DA90D910DE037A1F9E7B4
:10AA60006146019B009AFAF759FB0E9B8C469B5C52
:10AA70000D9A521E0D92137061460143F0D10D984C
:10AA800005A9081A20300190600703D501200004B1
:10AA9000844300E001270198874201DD381A00E075
:10AAA0000020019900904118029809180498401A52
:10AAB0000490E00306D421461A9B199A049800F0EA
:10AAC000B3F94519002706E003A81A9AC05D199941
:10AAD00090476D1C7F1C02988742F5DBE0030CD584
:10AAE00021461A9B199A049800F09EF9451904E032
:10AAF0001A9A3020199990476D1C0099481E0090B1
:10AB00000029F5DC08E00D980D990078491C0D919D
:10AB10001A9A199990476D1C0199481E01900029B5
:10AB2000F1DC63E109280100303132333435363746
:10AB30003839616263646566000000003031323389
:10AB40003435363738394142434445460000000029
:10AB500000F05AF94519761C3078002800D0E2E55B
:10AB600028461BB0F0BD600700D406271898C01D0A
:10AB7000C108C90048680A680831C30FDB0718918B
:10AB8000190001D09CA108E0210501D59BA104E09A
:10AB9000E10701D09AA100E09AA1430011985B0857
:10ABA000109165280CD006DC452809D046281DD018
:10ABB000472841D141E0662818D067283CD13CE0C5
:10ABC0000021112F01DB112000E0781C0191009081
:10ABD00008A911A8FFF7E8FC139905910021119A23
:10ABE00015927F1C12980197009150E00120C00738
:10ABF00003900120019008A9009711A8FFF7D4FC49
:10AC0000139A149905920022119B009212981593A1
:10AC1000059A0192002901D0104602E0791C4018E3
:10AC20000190381A01D5019804E04042401E00907E
:10AC3000781C0190C01B029043E0012F00DA01272D
:10AC40000021112F01DD112000E038460191009014
:10AC500008A911A8FFF7A8FC13990591119A0021E2
:10AC6000129815920091019721070CD40599B942C9
:10AC700001DB019900E00191012904DD159A491ECB
:10AC8000515C302906D0B84201DA011D05DA0121F4
:10AC9000029115E00199491EEDE7002805DC0099B5
:10ACA000411800910199091A03E0019A411C91424F
:10ACB00000DD01910099401A401C02900120C0075C
:10ACC0000390200706D402990198814202DB0020FC
:10ACD000C043029000206946C87707AF012103985E
:10ACE0000337C907884224D0022011902B201290EC
:10ACF000039800280CDA404203902D20129007E0C0
:10AD00000A210398FAF7F4F930317F1E0390397065
:10AD10001199481E11900029F2DC03980028EFD108
:10AD2000791E129808703078202108404530BF1EE7
:10AD3000387006A8C01BC01D03901098007800282A
:10AD400000D00120019941180298C01709180398F2
:10AD500009180498401A401E0490E00306D42146C6
:10AD60001A9B199A049800F05FF84519109800781A
:10AD7000002803D01A9A199990476D1CE00324D536
:10AD800021461A9B199A049800F04EF845191CE0C8
:10AD90000098002807DB00990598884203DD159884
:10ADA000405C199901E0199930201A9A904700984F
:10ADB0006D1C401C00900298401E0290002804D197
:10ADC0001A9A2E20199990476D1C0199481E0190DE
:10ADD0000029DDDC05E038781A9A7F1C1999904724
:10ADE0006D1C0399481E03900029F4DC21461A9B30
:10ADF000199A0498ACE600002D0000002B0000001A
:10AE00002000000000000000F8B5044600251E46A2
:10AE10001746880404D405E039462020B0476D1C4D
:10AE2000641EF9D52846F8BDFFB50446002581B05B
:10AE30001E46C80301D5302700E02027880404D52A
:10AE400005E038460399B0476D1C641EF9D52846C5
:10AE500005B0F0BDF8B54A002B4B520DD6182B4A61
:10AE60000C460546142E2BDA002E12DA284BFAF780
:10AE70004DFA00221346FAF779FC40D2002C03DA8F
:10AE80000124E40700253AE02046284337D0214C2E
:10AE900014E0214F0B46F7403B402B4331D01C4B75
:10AEA000FAF734FA00221346FAF760FC27D2002C96
:10AEB00003DD01200005F0400419BC4300251EE01D
:10AEC000332E1EDC33460027143BFF43DF4038425D
:10AED00017D00F4BFAF7C4FA00221346FAF746FCD4
:10AEE0000DD2002C0ADD142E0CD03420811B012041
:10AEF00088404019A84200D2641C0546BD43214643
:10AF00002846F8BD641CF9E701FCFFFF9C7500882A
:10AF10003CE4377E0000F03FFFFF0F007D2110B5BD
:10AF2000C900484300F001F810BD002140E000BF17
:10AF300000BF00BF00BF00BF00BF00BF00BF00BF19
:10AF400000BF00BF00BF00BF00BF00BF00BF00BF09
:10AF500000BF00BF00BF00BF00BF00BF00BF00BFF9
:10AF600000BF00BF00BF00BF00BF00BF00BF00BFE9
:10AF700000BF00BF00BF00BF00BF00BF00BF00BFD9
:10AF800000BF00BF00BF00BF00BF00BF00BF00BFC9
:10AF900000BF00BF00BF00BF00BF00BF00BF00BFB9
:10AFA00000BF00BF00BF00BF00BF00BF00BF491C03
:10AFB0008142BCD370470000FEB5044600200190DA
:10AFC00000906079734940000E5A61782578491ED7
:10AFD0007148CFB20163042D77D0072D75D00021C1
:10AFE0000291217801736C49E37901229205896904
:10AFF000002B6CD0914381616748217A4173217A9B
:10B0000082698907890B0A4382610021042000F0CC
:10B0100034FB324661492E2000F024FB3846FFF70E
:10B020000FFA5F4E0522705D810040185D4943189C
:10B0300007212B2000F030FB5B49029801220B18FE
:10B040000B21282000F028FB705D584980000A5829
:10B050000C21282000F011FBE079554980004018B0
:10B06000A1794900425A0221272000F0FBFA5148F9
:10B070007E00825B0421272000F0F4FAE0790028AA
:10B0800029D0A07804282CD02820694608722022D4
:10B090000621272000F0E6FA02AB01222621272014
:10B0A00000F0FAFA444938014018E1788900425822
:10B0B0000821272000F0E1FAA17A601C627A0902D7
:10B0C000114313D016E000E001E0012188E71143AD
:10B0D000F608816190E764220621272000F0C2FA79
:10B0E000E0E71020694608720246D1E73349017251
:10B0F000090A4172417A007A0A020243202127207C
:10B1000000F0B0FA2E4F0C2123203A6800F0B5FA77
:10B11000F01982880421232000F0A4FAA0790028E5
:10B120000BD0E0792749012243180021212000F0AB
:10B13000B3FA03200190012000902A07120F10019A
:10B140000243607800218007000B0243019800054C
:10B1500002430098400402432079C006400902439C
:10B160006079C00602431F2000F087FAA07861785A
:10B170000123084302040848DB030261E179490323
:10B1800019430A4302610021082000F076FA0020EA
:10B19000FEBD0000ECBA00083001002004280000C9
:10B1A00094BA00080C0000202A0000209CBA000875
:10B1B000BCBA0008C8BA0008CCBA000841100000A8
:10B1C000B4BA00082C00002038B50C4607498A8B19
:10B1D000002102432C2000F045FA684604706B46BB
:10B1E000012206212C2000F057FA38BD3001002042
:10B1F00010B5FFF712F910BD10B504460421362032
:10B2000000F0FCF80121C902002C01D0084300E045
:10B21000884302460421362000F02FFA10BD0000BA
:10B2200038B540206946087000210E2000F0E6F88D
:10B230000446002211460E2000F01FFA6B46012240
:10B2400000210D2000F028FA074A00210F2000F00D
:10B2500014FA00F0EDF9224600210E2000F00DFA5C
:10B2600002480021017338BDF8FF27245001002057
:10B27000FEB50546042069460870514C00206075F3
:10B2800021462031206348710873A0836063A06366
:10B2900000F0C8F84B4E206002E000F0C3F82060D8
:10B2A000B042FAD10020FFF7E9F800F0BBF8464EB3
:10B2B00020603078242801D9243806E00621F9F7E7
:10B2C00017FF0622101A40010843020601040A4330
:10B2D00001020A430243B260706000211E2000F0A8
:10B2E000CCF900F09FF820606B4601220021242059
:10B2F00000F0D2F91E20FFF735F986B2300AA073AC
:10B300000420FFF72FF9074600F08CF8206038067C
:10B31000000E0DD002206946087101AB01221221F6
:10B320002D2000F0B9F9A08B012109030843A08367
:10B3300000F078F820600620FFF714F9606007201D
:10B34000FFF710F9A060F006C00E207501D11020A3
:10B350002075C0B200F0DCF9E80707D0FFF7E9F884
:10B36000A08B0121C9020843A0830AE005213620F1
:10B3700000F02EF81549084002460521362000F05D
:10B3800071F90120FFF77AF80021042000F036F867
:10B39000A0610021262000F031F81521890308431F
:10B3A00002460021262000F068F9002226213620DE
:10B3B00000F058F900F036F820600020FEBD0000D3
:10B3C000300100203001CADE00000020FFFD000037
:10B3D00038B5094C89B280B26B46022200F028F8D9
:10B3E000002806D1684640780102684600780818AF
:10B3F00084B2204638BD0000FFFF000038B50024AD
:10B40000E44389B280B26B46042200F011F80028B0
:10B4100006D103216846435C2202D418491EFAD59E
:10B42000204638BD10B500210846FFF7E7FF10BDE4
:10B4300038B5002909D0402420436C462070C8B29A
:10B440007F2906D8607002200AE069460870012052
:10B4500006E0802420436C466070C809A070032079
:10B46000694600F0B7FA38BD10B5144603460A46DF
:10B4700021461120FFF7DCFF10BD10B50346052261
:10B4800000211520FFF7D4FF10BD10B5034605229B
:10B4900000211720FFF7CCFF10BD38B5054600206E
:10B4A0006946087000F0C4F8FF2401342246002DDC
:10B4B00001D00322120200210D2000F0D3F8002D4C
:10B4C00013D06B46012203210F20FFF7B1FF68461E
:10B4D0000078000709D5FFF7A3FE224600210D20C2
:10B4E00000F0C0F80020C04338BD002038BD10B5C2
:10B4F000024601210A2000F0C0F810BD10B5044634
:10B5000000211A20FFF77AFF000D22030005120B1D
:10B51000024300211A2000F0B0F810BD10B5024619
:10B5200002492E2000F09EF810BD00000418000013
:10B53000F8B505466B46012203210420FFF778FF8A
:10B540000126114C3607002D0DD02A4600210C2073
:10B5500000F088F8694608781021084369460870A9
:10B56000A069304307E069460878EF210840694642
:10B570000870A069B0430B46A0610122032104209A
:10B5800000F08AF8F8BD00003001002010B5024636
:10B590000021182000F066F810BD0000F8B507463D
:10B5A000002568460570B807204C2E4600280ADAA8
:10B5B0008020694608706B46012200210D2000F0B2
:10B5C0006BF801202073F8076946087821D006211E
:10B5D0000843694608706B46012200210D2000F0E7
:10B5E0005BF803210F20FFF7F3FE8121C900084219
:10B5F00019D04020694608706B46012200210D20B9
:10B6000000F04AF80020FFF7F7FD00252673ED4310
:10B6100009E002210843694608706B4601220021B7
:10B620000D2000F039F82846F8BD00005001002038
:10B630001CB56B46012203210F20FFF7F9FE684677
:10B6400000784022C1091040C9014000814208D061
:10B65000012069460871024601AB03210D2000F06C
:10B660001BF81CBD08B56B461A70120A5A7089B2D5
:10B6700080B2022200F010F808BD38B500236C46F5
:10B68000E254120A5B1C042BFADB89B280B2234617
:10B69000042200F001F838BD38B58024002909D013
:10B6A000C02528436D462870C8B27F2907D8687026
:10B6B000022009E0204369460870012004E020438D
:10B6C0006870C809A8700320694600F0BFF938BD4A
:10B6D00010B51446012312189B029A4202D9002089
:10B6E000C04310BD0B46821E21460920FFF7D4FF40
:10B6F000002010BD10B5054A8905126901430A43AF
:10B7000000210820FFF7B9FF002010BD3001002004
:10B7100038B504466B4601220E212B20FFF788FE28
:10B7200068460078E10640094001C90E01436846B9
:10B7300001706B4601220E212B20FFF7ADFF38BDB3
:10B7400010B5002142541C06120A22431B0A491C50
:10B750000429F7DB10BD000013B501231A46694622
:10B760000248FCF765FC00981CBD00005C15002039
:10B770007CB5002425466846FFF77FFE0420694615
:10B78000220E2D02154322020C5C1443401EF7D5F5
:10B79000204629467CBD7CB5002425466846FFF737
:10B7A00074FE04206946220E2D02154322020C5C11
:10B7B0001443401EF7D5204629467CBDFBF720F9EF
:10B7C000FDF7D8FFFCF7EEFF40494148002522C0B5
:10B7D00005608561C5613F490562C1600838FBF7B6
:10B7E0009FFAFCF7CBFFFDF7E3F8FDF77FF8FCF7D6
:10B7F00091FF052601223607D1033046FBF7EBF80F
:10B80000FDF726FDFCF77AFEFAF7C0F9FAF78EF994
:10B81000FCF780FC0721B015FFF7D6FC2E4C0A215F
:10B82000208A01224843608411033046FBF7D3F895
:10B830002748C8222949C830FCF7C8FB284F294EA1
:10B84000207900283FD0607800283CD0FDF792FF97
:10B850002571FAF787FB20700F280AD901221103FE
:10B860003046FBF7B8F8FEF7D3F8002201210903B0
:10B8700009E0012251033046FBF7ADF8FEF7C8F8A6
:10B880000022012149033046FBF7A5F8FCF762FDD1
:10B89000608C002801D0401E60841348618C0078C1
:10B8A0000843CDD13878002801D00328C8D1012120
:10B8B000C9023046FBF782F80028C1D101210846B1
:10B8C000FBF742FBBCE7FCF745FDB9E7007C004015
:10B8D00094140020FFFF0000D4000020940C0020EE
:10B8E00069000020000400504200002010B586B01E
:10B8F0001748FBF798F914216846F9F758FC1548E2
:10B900000090032001900020029005206946000766
:10B91000FAF798FF69461048FAF794FF69460F480E
:10B92000FAF790FF01210846FBF70EFBFF240134D4
:10B930002046FBF7E1FA0A49086804221043086030
:10B940002046FBF7E9FAFBF7EFFA06B010BD00005E
:10B9500094140020FFFF0000000400500008005075
:10B960000070004010B50122920217491748FAF7FB
:10B9700099F91548164902888A4223D00180FF218F
:10B9800001318180FF21F531C1800A21018100212F
:10B990001E224181D24382810122C28181831E23E2
:10B9A000C38602230387782343878287C2870246A0
:10B9B0004032118451849184C18391801421818209
:10B9C00000F02EF810BD00005C0D002000FC000807
:10B9D000AA550000F0B58C46002510260521090760
:10B9E0008E620E4C08E067467F5DE760A768FF0740
:10B9F000FCD0E7681F706D1C8542F4DB0020074611
:10BA000006E0E760A568ED07FCD0E5681D54401C22
:10BA10009042F6D38E610020F0BD0000003001405E
:10BA200070B572B60124074DA40221462846FAF7E4
:10BA30001FF9002804D0224603492846FAF7BCF92A
:10BA400062B670BD00FC00085C0D0020F0B500255A
:10BA5000102605279C463F070B46BE620C4C06E0AD
:10BA6000595DE160A168C907FCD0E1686D1C8542A1
:10BA7000F6DB002007E06146095CE160A168C907C8
:10BA8000FCD0E168401C9042F5D3BE610020F0BDBF
:10BA9000003001400000010203040005405C00008A
:10BAA000A05C0400C06C0800805C0400E03F1E0045
:10BAB000E07D1E0007A9022570889B880A001600F9
:10BAC000010006000100020087008D002D001A31E0
:10BAD00052001A339A001A351D011A376B003B3198
:10BAE000BE003B335E013B3596023B37000099595F
:10BAF0009959EB518F421E45142E0080EB51F528C9
:10BB00003333E13A703DE13AC235852BC2353333E8
:10BB1000C235C235AE47E13A5138A3305138000042
:10BB200000000000000001020304060708090304E6
:10BB300006080C1018203000000000010203040069
:10BB400060BB00080000002030010000EC59000834
:10BB5000A0BB000830010020581900000CA4000808
:10BB6000C1130704380D091E0805400826091040B6
:10BB700008560A131D043B08BE0516D8BC40100821
:10BB800052010334C84203525C121B0202B514096D
:10BB90000102628149A00146294C92045220000012
:04000005080050C1DE
:00000001FF
